:100000008015FFFFFFFFFFFFFFFFFF0200F3FFFF71
:10001000FFFFFFFFFFFFFF12020385A020A2009257
:100020000FA201920EA202920DA203920CA20492C0
:100030000BA205920AA2069209A2079208852160E6
:100040007580FF858061E5B0540724028380080233
:10005000050B161C2D3870F562E5B0540724028399
:100060008008D0A0408020004080F563757408753A
:100070007500757600757808757900757A00859039
:100080007275A882857071857404857505857606FC
:100090008562078563001201A985600485610512E8
:1000A00001D3EB54062402838008000001010303FE
:1000B00002025371FC427130B530857804857905B0
:1000C000857A068562078563001201A9856004852B
:1000D00061051201D3EB540624028380080000045A
:1000E000040C0C08085371F342714371F085719050
:1000F000020084C0E0C0F0C0D0859070E5700303BA
:10010000540CF5F0E572C4540345F02402838010CA
:1001100000030100010000030300000100010300CF
:1001200010E116F5F0E57625F0F576E5753400F585
:1001300075E5743400F5748013C3E5769401F576A3
:10014000E5759400F575E5749400F57430B550E5E7
:1001500070C4540CF5F0E5722323540345F02402D7
:100160008380100003010001000003030000010070
:1001700001030010E116F5F0E57A25F0F57AE5794E
:100180003400F579E5783400F5788013C3E57A9486
:1001900001F57AE5799400F579E5789400F57885AC
:1001A0007072D0D0D0F0D0E032E4F9FAFB75F00CE8
:1001B000C3EB33FBEA33FAE933F9E833F8EF33FF03
:1001C000500DEB2EFBEA3DFAE93CF9E83400F8D596
:1001D000F0DE227F18C37E00EB33FBEA33FAE9330B
:1001E000F9E833F8EE33FEC3E89DF8EE9CFE5006C6
:1001F000E82DF8EE3CFEB3DFDFEB33FBEA33FAE940
:1002000033F9225389F0438902758C8330B5037525
:050210008C06D28C22D7
:00000001FF
